:020000040800F2
:1000000000000120DD270008A1250008A325000825
:10001000A5250008A7250008A92500080000000064
:10002000000000000000000000000000AB250008F8
:10003000AD25000800000000AF250008B12500082C
:10004000252800082528000825280008252800085C
:10005000252800082528000825280008252800084C
:10006000252800082528000825280008252800083C
:100070002528000825280008B5250008C125000806
:10008000252800082528000825280008252800081C
:10009000252800082528000825280008252800080C
:1000A00025280008252800082528000825280008FC
:1000B00025280008252800082528000825280008EC
:1000C00025280008252800082528000825280008DC
:1000D00025280008CD250008252800082528000827
:1000E00025280008252800082528000825280008BC
:1000F00025280008252800082528000825280008AC
:10010000252800082528000825280008252800089B
:100110002528000825280008D925000825280008DA
:10012000252800082528000825280008252800087B
:1001300000000000000000000000000000000000BF
:1001400000000000000000000000000000000000AF
:10015000000000000000000000000000000000009F
:10016000000000000000000000000000000000008F
:10017000000000000000000000000000000000007F
:10018000000000000000000000000000000000006F
:10019000000000000000000000000000000000005F
:1001A000000000000000000000000000000000004F
:1001B000000000000000000000000000000000003F
:1001C000000000000000000000000000000000002F
:1001D000000000000000000000000000000000001F
:0401E0005FF8E0F1F3
:1001E40010B5054C237833B9044B13B10448AFF36D
:1001F40000800123237010BD800200200000000055
:10020400D838000808B5034B1BB103490348AFF3C2
:10021400008008BD0000000084020020D8380008D7
:10022400D0400B1CD1409C46203AD3401843524244
:10023400634693401843704738B50E4B054618780B
:100244004FF47A73B3FBF0F30B4A1068B0FBF3F08E
:1002540000F08CF8044658B90F2D09D802462946F7
:100264004FF0FF3000F042F8044B20461D6038BDCB
:10027400012038BD000000201802002004000020E6
:10028400074A08B51368032043F01003136000F015
:100294001BF80020FFF7D0FF02F0ACF8002008BDE7
:1002A40000200240034A044B11681B780B4413607E
:1002B400704700BF2407002000000020014B18688D
:1002C400704700BF24070020074A0002D36800F4E7
:1002D400E06023F4E0631B041B0C43F0BF6343F4AE
:1002E40000330343D360704700ED00E0174B30B593
:1002F400DC68C4F30224C4F10703251D042B28BFC2
:100304000423062D4FF0010598BF002405FA03F3DA
:1003140003F1FF3388BF033C1940A14005FA04F4FC
:10032400013C2240002842EA01024FEA0212AFBF18
:1003340000F16040064B00F00F00D2B2A5BFD2B26C
:1003440000F561401A5480F8002330BD00ED00E050
:1003540014ED00E00123420900F01F0003FA00F04D
:10036400014B43F82200704700E100E00138B0F18E
:10037400807F0AD2F021064B064A586082F8231087
:100384000020072298601A6070470120704700BF60
:1003940010E000E000ED00E010B5002832D0016864
:1003A400194B1424994225D8184AA3F207430A4446
:1003B400B2FBF4F2920002648468C36343680A687F
:1003C4002343C46822F47F522343046922F0300299
:1003D40023434469234384692343C4692343134364
:1003E4000B600122002380F82120836380F82030F1
:1003F400184610BD064B0B44B3FBF4F39B00036497
:10040400044BD9E7012010BD07040240F8FFFDBFEB
:10041400F8FBFDBF00040240F0B590F82040012C29
:1004240035D0012490F8215080F82040A5424FF0A7
:1004340000064FF0020428D180F821400468866346
:100444002668076C26F001062660C66BBD40756001
:10045400636043680568102BC36A0BBFA260A16088
:10046400E160E2604BB1236843F00E0323602B6824
:10047400002043F001032B60F0BD236823F0040344
:100484002360236843F00A03F0E780F82060022029
:10049400F0BD000090F8213010B5022B03D00423E6
:1004A4008363012010BD03681A6822F00E021A60EB
:1004B4001A6822F001021A60294A934224D902F5EB
:1004C4006272934219D01432934218D01432934278
:1004D40017D0143293420CBF4FF480534FF480333F
:1004E400204A53600123002480F82130436B80F8B4
:1004F40020409BB39847204610BD0123F0E710230A
:10050400EEE74FF48073EBE717498B4216D01431B2
:100514008B4215D014318B4214D014318B4214D039
:1005240014318B4214D014318B4214D0934214BF33
:100534004FF480334FF080730C4AD2E70123FBE77A
:100544001023F9E74FF48073F6E74FF48053F3E791
:100554004FF48033F0E74FF48013EDE7184610BDF5
:1005640080000240000402400800024000000240F3
:1005740070B40425C66B026C346803689540254248
:10058400196855D04D0753D51A6896065EBF1A6888
:1005940022F004021A60604A93421FD902F5627283
:1005A400934214D01432934213D01432934212D093
:1005B400143293420CBF4FF480434FF48023574AC4
:1005C4005360C36A002B00F0A58070BC1847042355
:1005D400F5E74023F3E74FF48063F0E750498B429B
:1005E40016D014318B4215D014318B4214D01431EF
:1005F4008B4214D014318B4214D014318B4214D05A
:10060400934214BF4FF480234FF08063454AD7E7E9
:100614000423FBE74023F9E74FF48063F6E74FF444
:100624008043F3E74FF48023F0E74FF48003EDE7D2
:1006340002259540254257D08D0755D51A68940652
:1006440006D41A6822F00A021A60012280F82120D6
:10065400314A93421ED902F56272934213D0143286
:10066400934212D01432934211D0143293420CBFED
:100674004FF400534FF40033284A5360002380F8AA
:100684002030836A9EE70223F6E72023F4E74FF441
:100694000073F1E722498B4216D014318B4215D0F6
:1006A40014318B4214D014318B4214D014318B4248
:1006B40014D014318B4214D0934214BF4FF400333E
:1006C4004FF00073174AD8E70223FBE72023F9E72A
:1006D4004FF40073F6E74FF40053F3E74FF400339D
:1006E400F0E74FF40013EDE708259540254211D0BB
:1006F40009070FD5196821F00E011960012303FAC7
:1007040002F27260836380F82130002380F8203085
:10071400036B57E770BC704780000240000402403E
:100724000800024000000240114AD36813F010038D
:1007340005D01049CB6943F00203CB611023D26882
:10074400500706D50B4943F00403CA6942F001027D
:10075400CA61074AD169C90708D50648C16941F089
:100764000401C161D16921F00101D161D3607047F5
:100774000020024028070020064B186910F0800072
:1007840007D0054A5A6002F188325A601869C0F3EA
:10079400C01070470020024023016745034A00202F
:1007A400136943F080031361704700BF00200240C7
:1007B400F8B50646FFF782FD114C07462546E36867
:1007C400D80712D4E368990644BF2023E360EB689A
:1007D400DA0606D4EB69DB0703D4E86810F00400FA
:1007E40002D0FFF7A1FF0120F8BD731CE7D00EB9BA
:1007F4000320F8BDFFF762FDC01B8642DFD2F7E796
:10080400002002402DE9F84F1F4C9946237E0546EF
:10081400012B0F46904633D001234CF250302376FF
:10082400FFF7C6FF40BB012D03D0022D0CBF0225EC
:1008340004250026B246DFF854B03201404649464A
:10084400FFF7EEFCC4F81CA0DBF8103080B243F0D4
:100854000103CBF8103027F816004CF25030FFF7A4
:10086400A7FFDBF8103023F00103CBF8103018B9E0
:100874000136F3B29D42E0D800232376BDE8F88F19
:100884000220BDE8F88F00BF2807002000200240A6
:100894000022064BDA61064B1A6942F004021A611F
:1008A4001A6942F040021A61704700BF280700200D
:1008B400002002400022064BDA61064B1A6942F01E
:1008C40002021A6158611A6942F040021A617047C3
:1008D40028070020002002402DE9F041234D07465F
:1008E4002B7E8846012B3DD0012403682C76022BF5
:1008F4004CF2503013D1FFF75BFF20B101200023ED
:100904002B76BDE8F081FFF7C3FF4CF25030FFF7C0
:100914004FFF174A136923F004031361EFE7FFF74E
:1009240047FF0028EAD14FF0FF33C8F800302046D3
:10093400BE680F4CFA68BB6803EBC2239E42DED24A
:100944003046FFF7B7FF4CF25030FFF731FF236911
:1009540023F00203236110B1C8F80060CFE706F565
:100964000066E7E70220BDE8F08100BF2807002009
:10097400002002402DE9F74F002216466C4F6D4BC4
:10098400DFF8B8E1DFF8B8C14FF001080C6808FAE5
:1009940006F808EA0404A04540F085804D68122D4D
:1009A40000F0B78000F28D80022D00F0AF8000F2DD
:1009B4008180002D00F09180012D00F0A5804FF082
:1009C4000F09FF2C93BF824606F18045083DD0F8FD
:1009D40000B092BFB500D0F804B0AD0009FA05F834
:1009E4002BEA080802FA05F588BF00F1040A48EA70
:1009F4000505CAF80050D1F804A01AF0805F52D05F
:100A0400BD6926F0030845F00105BD61BD6908F123
:100A1400804805F00105019508F5803806F0030BC0
:100A2400019D4FEA8B0BD8F8085009FA0BF925EA17
:100A34000909414DA84271D005F58065A8426FD0DF
:100A440005F58065A8426DD005F58065A8426BD098
:100A540005F58065A84269D070450CBF05250625BB
:100A640005FA0BF545EA0905C8F808501D681AF49B
:100A7400803F14BF2543A5431D605D681AF4003F01
:100A840014BF2543A5435D609D681AF4801F14BFFD
:100A94002543A5439D60DD681AF4001F14BF2C4351
:100AA40025EA0404DC600136102E7FF46DAF03B038
:100AB400BDE8F08F032D25D0112D80D1CA680432F2
:100AC4007DE7654509D012D8DFF878904D4504D00C
:100AD40009F580394D457FF472AF8A68E2B1012A85
:100AE4000CBFC0F81080C0F81480082267E7DFF854
:100AF40058904D45F1D009F580394D45EDD0A9F513
:100B04008019E7E700225AE7CA6858E7CA6808323A
:100B140055E7CA680C3252E7042250E700259FE7E4
:100B240001259DE702259BE7032599E7042597E71F
:100B3400001002400004014000080140001C014074
:100B44000000211000001110000031100AB10161F1
:100B540070470904FBE7C3685940C160704700004F
:100B640038B5044608B9012038BD90F83D3003F08B
:100B7400FF021BB980F83C2001F05EFC24232268AC
:100B840084F83D30136823F00103136000F0E2FAA7
:100B940063682F4A934230D82E4A9042E3D92E4AB2
:100BA4002168B0FBF2F24A6001320A62284A013835
:100BB400934232D85B00B0FBF3F0431CC3F30B0346
:100BC400042B38BF0423CB61226AE369002013435A
:100BD4000B60E268236913438B60A2696369134362
:100BE400CB600B6843F001030B602023206484F87E
:100BF4003D30206384F83E0038BD184A9042B2D993
:100C0400154D4FF49672B0FBF5F521686A434D60BB
:100C14004FF47A75B2FBF5F2C6E7A26852B903EB5A
:100C24004303B0FBF3F0431CC3F30B036BB143F476
:100C34000043C8E719225343B0FBF3F0431CC3F34A
:100C44000B0313B143F44043BDE70123BBE700BFEB
:100C5400A08601007F841E0040420F00FF083D0073
:100C640003682DE9F341DB07054610D42B689F0781
:100C74005ED42B68190700F195802B685A0700F1A0
:100C8400BF80EA69002A40F02D81002014E0904CD6
:100C9400636803F00C03042B07D0636803F00C03B0
:100CA400082B0CD16368DE0309D523689C03DDD5CA
:100CB4006B68002BDAD1012002B0BDE8F0816B68CB
:100CC400B3F5803F10D1236843F480332360FFF7EA
:100CD400F5FA064623689803C8D4FFF7EFFA801B99
:100CE4006428F7D90320E7E79BB9236823F480330A
:100CF4002360236823F480232360FFF7DFFA06468A
:100D040023689903B2D5FFF7D9FA801B6428F7D971
:100D1400E8E7B3F5A02F236803D143F480232360CD
:100D2400D1E723F480332360236823F48023CDE7C1
:100D3400674C636813F00C0F07D0636803F00C036F
:100D4400082B10D16368DA030DD423689B0702D5FE
:100D54002B69012BAFD123686A6923F0F80343EAB6
:100D6400C203236085E72A695A4B6AB101221A60DB
:100D7400FFF7A4FA064623689F07ECD4FFF79EFA10
:100D8400801B0228F7D9ADE71A60FFF797FA0646E9
:100D9400236898077FF56DAFFFF790FA801B022850
:100DA400F6D99FE7AA694A4C4B4BDAB101221A6083
:100DB400FFF784FA0646636A9B070DD54FF4FA528F
:100DC400464B1B68B3FBF2F3019300BF019B5A1E11
:100DD4000192002BF9D150E7FFF770FA801B02282B
:100DE400E9D97FE71A60FFF769FA0646636A9F0745
:100DF4007FF543AFFFF762FA801B0228F6D971E74B
:100E0400334CE369D80024D40127E36943F08053C9
:100E1400E361E36903F080530093009B304E336831
:100E2400D90518D5EB68012B26D1236A43F00103B9
:100E34002362FFF743FA41F288368046236A9B0710
:100E44003FD5002F3FF41DAFE36923F08053E361E6
:100E540017E70027E2E7336843F480733360FFF752
:100E64002DFA80463368DA05DCD4FFF727FAA0EBC5
:100E740008006428F6D935E7ABB9236A41F288380B
:100E840023F001032362236A23F004032362FFF7A0
:100E940015FA0646236A9807D3D5FFF70FFA801B85
:100EA4004045F7D91EE7052B236A03D143F0040319
:100EB4002362BAE723F001032362236A23F00403C5
:100EC400B6E7FFF7FBF9A0EB0800B042B6D909E793
:100ED40000100240000042428004424218020020F6
:100EE40000700040224C636803F00C03082B3FF4AD
:100EF400E2AE00231F4E022A33602BD1FFF7DEF946
:100F04000746236899011FD42B6AB3F5803F05D1A6
:100F14006268A96822F400320A436260696A6268FE
:100F24000B4322F474121343636001233360FFF70D
:100F3400C5F9054623689A013FF5A7AEFFF7BEF948
:100F4400401B0228F6D9CDE6FFF7B8F9C01B0228EA
:100F5400D7D9C7E6FFF7B2F9054623689B017FF5A9
:100F640094AEFFF7ABF9401B0228F6D9BAE600BFEE
:100F7400001002406000424230B5194B87B002AC09
:100F840003F11005224618685968083303C2AB42BE
:100F94001446F7D101238DF80430022311498DF84A
:100FA40005304B6803F00C02082A17D1C3F38342BF
:100FB40006A80244DB0312F8102C0CD54B680A482F
:100FC400C3F34043504306AA134413F8143CB0FB44
:100FD400F3F007B030BD05485043FAE70248F8E79C
:100FE400F03800080010024000127A0000093D00A9
:100FF400544A2DE9F0411368054603F007038B4278
:101004000E462AD329688C0734D4CA0747D44D4ADC
:10101400136803F007039E42C0F082802A684A4C9A
:1010240012F0040F40F08780130706D563682A691D
:1010340023F4605343EAC2036360FFF79DFF6368D0
:10104400424AC3F30313D35CD840414B18600020D9
:10105400FFF7F2F80020BDE8F081136823F00703DE
:101064000B431360136803F007039942CAD00120AD
:10107400BDE8F081344B11F0040F1EBF5A6842F4EE
:10108400E0625A60080742BF5A6842F460525A60EC
:101094005A68A86822F0F00202435A60B5E76A6809
:1010A400294C012A23681CD113F4003FDFD0636864
:1010B40041F2883823F0030313436360FFF7FEF81B
:1010C4006B680746012B14D1636803F00C03042BEF
:1010D4009DD0FFF7F3F8C01B4045F5D90320BDE8C8
:1010E400F081022A02D113F0007FDFE713F0020F30
:1010F400DCE7022B0FD1636803F00C03082B86D0C6
:10110400FFF7DCF8C01B4045F5D9E7E7FFF7D6F851
:10111400C01B4045E2D8636813F00C0FF6D176E7A4
:10112400136823F0070333431360136803F00703C2
:101134009E429CD172E76368E96823F4E0630B4341
:10114400636071E70020024000100240F63A000894
:1011540018020020044B054A5B68C3F30223D35CE6
:10116400034A1068D840704700100240063B00084C
:1011740018020020044B054A5B68C3F3C223D35C06
:10118400034A1068D840704700100240063B00082C
:101194001802002003680020DA6842F00102DA60D5
:1011A4001A6842F001021A6070477047704770472E
:1011B4007047036810B51A69044691070ED5DA68BA
:1011C40092070BD56FF002021A6101229B69027724
:1011D4009B0777D0FFF7EAFF0023237723681A6978
:1011E400500710D5DA6851070DD56FF004021A6163
:1011F40002229B69227713F4407F204668D0FFF7D0
:10120400D5FF0023237723681A6912070FD5DA68FC
:1012140010070CD56FF008021A610422DB692277EB
:10122400990720465AD0FFF7C1FF0023237723688C
:101234001A69D20610D5DA68D0060DD56FF01002FF
:101244001A610822DB69227713F4407F20464BD0D1
:10125400FFF7ACFF0023237723681A69D10708D569
:10126400DA68D20705D56FF0010220461A6100F052
:101274008DFF23681A69100608D5DA68110605D5AA
:101284006FF0800220461A6100F0BFF823681A69E3
:10129400520608D5DA68500605D56FF0400220469C
:1012A4001A61FFF785FF23681A69910622D5DA6867
:1012B40092061FD56FF020022046BDE810401A6147
:1012C40000F0A2B8FFF771FF2046FFF770FF83E735
:1012D400FFF76BFF2046FFF76AFF92E7FFF765FF12
:1012E4002046FFF764FFA0E7FFF75FFF2046FFF704
:1012F4005EFFAFE710BD0000244A0368904212D09D
:1013040002F5006290420ED0B0F1804F0BD0A2F5EE
:101314009832904207D002F58062904203D002F5E1
:10132400806290421DD14A6823F070031343174A28
:10133400904212D002F5006290420ED0B0F1804F7C
:101344000BD0A2F59832904207D002F58062904209
:1013540003D002F58062904203D1CA6823F440733B
:1013640013434A6923F08003134303608B68C36209
:101374000B688362054B984203D003F500639842DF
:1013840001D10B690363012343617047002C0140C1
:1013940010B50446A0B190F83D3003F0FF021BB92C
:1013A40080F83C2001F07AF80223206884F83D306C
:1013B400211DFFF7A1FF0123002084F83D3010BD5B
:1013C400012010BD90F83C3010B5012B4FF0020302
:1013D40018D080F83D3003680C685A68496822F0D8
:1013E40070025A605A6822435A609A6822F0800256
:1013F4009A609A680A439A60012380F83D3000237A
:1014040080F83C30184610BD704770470368DA68AE
:1014140022F49072DA605A6922F001025A612023A0
:1014240080F83A30704700002DE9F0470568C2683B
:101434002B69016923F4405313432B618368EA68E1
:101444000B43416922F4B05222F00C020B431343C4
:10145400EB606B69826923F4407313436B61404B07
:1014640081469D424FF0190446D1FFF783FE04FBE9
:1014740000F3D9F804604FF06408B600B3FBF6F348
:10148400B3FBF8F31E01FFF775FE6043D9F804308F
:101494009B00B0FBF3F7FFF76DFE6043D9F804300F
:1014A4009B00B0FBF3F3B3FBF8F308FB13731B01CE
:1014B4003233B3FBF8F303F0F007FFF75BFE60434E
:1014C400D9F804209200B0FBF2FAFFF753FE604310
:1014D400D9F804309B00B0FBF3F3B3FBF8F308FB3B
:1014E40013A31B013233B3FBF8F303F00F033B43A5
:1014F4003344AB60BDE8F087FFF72CFE04FB00F338
:10150400D9F804604FF06408B600B3FBF6F3B3FBFC
:10151400F8F31E01FFF71EFE6043D9F804309B0068
:10152400B0FBF3F7FFF716FE6043D9F804309B00D5
:10153400B0FBF3F3B3FBF8F308FB13731B01323373
:10154400B3FBF8F303F0F007FFF704FE6043D9F8A8
:1015540004209200B0FBF2FAFFF7FCFDB7E700BFEE
:1015640000380140F8B504460E4617461D4621686A
:101574000B6836EA030301D10020F8BD6B1CF7D0D9
:1015840095B923680320DA6822F4D072DA605A69C4
:1015940022F001025A61202384F8393084F83A3069
:1015A400002384F83830F8BDFEF788FEC01B85425E
:1015B400DDD2E6E710B5044640B390F8393003F0C5
:1015C400FF021BB980F8382000F07CFF2423226836
:1015D40084F83930D368204623F40053D360FFF7EE
:1015E40023FF236800201A6922F490421A615A6981
:1015F40022F02A025A61DA6842F40052DA602023A7
:10160400E06384F8393084F83A3010BD012010BD0D
:101614002DE9F0411F4690F839300446202B0D4641
:1016240090464ED1002949D0002A47D090F838304E
:10163400012B46D0012380F838300023C3632123D3
:1016440080F83930FEF73AFE0646A4F82480A4F860
:101654002680E38C9BB26BB93B4632464021204640
:10166400FFF780FFA8B9202384F8380084F83930C4
:10167400BDE8F081E38C3246013B9BB2E384A3686E
:101684008021B3F5805F20463B460ED1FFF76AFF09
:1016940010B10320BDE8F0812B882268C3F308034E
:1016A4005360236943B90235D3E7FFF75BFF002892
:1016B400EFD123682A785A600135CAE70120BDE8D2
:1016C400F0810220BDE8F08138B50446134694F851
:1016D4003920202A2AD139B333B394F83820012A87
:1016E40024D00122002584F838202122E384206BB1
:1016F400E56384F839200E4AA384216282620D4A8C
:101704004563C2620C4A026322680432FEF784FE17
:101714006FF04002236828461A605A6984F83850EA
:1017240042F080025A6138BD012038BD022038BD24
:10173400D317000801180008CD180008134690F8C4
:101744003A2073B5202A054638D1002934D0002B1D
:1017540032D090F83820012A30D00122002480F8B9
:101764003820222281628385C46380F83A20406B4A
:10177400134A2E688262134A4463C262124A0263A5
:101784000A46311DFEF748FE20462B6801941A686C
:1017940001925A6885F838400192019ADA6842F455
:1017A4008072DA605A6942F001025A615A6942F061
:1017B40040025A6102B070BD0120FBE70220F9E744
:1017C4000B180008C1180008CD180008704708B5A8
:1017D4000368426A1B6813F020030AD1D384136898
:1017E4005A6922F080025A61DA6842F04002DA60F3
:1017F40008BD1046FFF7EAFF08BD704708B5406A08
:10180400FFF7FBFF08BD08B50368426A1B6813F0C5
:10181400200310D1D3851368D96821F48071D9606D
:10182400596921F001015961596921F04001596157
:10183400202382F83A30104600F0A0FF08BD90F84B
:101844003A3010B5222B36D183680169B3F5805F35
:101854000268836A23D15268E9B9C2F3080223F803
:10186400022B8362C48D013CA4B2C4858CB9036885
:10187400DA6822F02002DA60DA6822F48072DA6030
:101884005A6922F001025A61202380F83A3000F0AC
:1018940075FF002010BDD2B223F8012BE1E721B976
:1018A400591C526881621A70DCE75268591C8162C3
:1018B40002F07F02F7E7022010BD704708B5406AC6
:1018C400FFF7FBFF08BD7047416A08B50B685A690A
:1018D40091F8390021280AD1120608D50022CA84B9
:1018E400DA6822F0C002DA60202281F839205B69CC
:1018F40091F83A20222A06D15B0604D50023084633
:10190400CB85FFF783FDCB6B084643F01003CB6315
:10191400FFF7D9FF08BD0000036870B51A680446D4
:101924001607D9685D6907D196065AD58D0658D52C
:10193400BDE87040FFF783BF15F0010502D111F433
:10194400907F4ED0D30705D5CE0542BFE36B43F05D
:101954000103E363500704D51DB1E36B43F00203B5
:10196400E363930704D51DB1E36B43F00403E3631E
:10197400160704D51DB1E36B43F00803E363E36B7F
:10198400002B66D0950604D5880602D52046FFF7BD
:1019940056FF236820465D69E26B110702D415F0F7
:1019A40040051AD0FFF732FD23685A69520610D554
:1019B4005A69606B22F040025A6150B1254B43636F
:1019C400FEF768FD002844D0606BBDE87040436BAF
:1019D40018472046FFF777FF70BDFFF774FFE563F4
:1019E40070BD160627D50D0625D594F83920212A71
:1019F4002FD1A268B2F5805F226A17D11188C1F392
:101A040008015960216979B902322262E28C013AF3
:101A140092B2E284EAB9DA6822F08002DA60DA6823
:101A240042F04002DA6070BD0132EEE7511C2162DF
:101A340012785A60EAE750060BD54A0609D5DA68E7
:101A4400204622F04002DA60202384F83930FFF780
:101A5400BDFE70BD5D1A000808B50023406AC38549
:101A6400C384FFF730FF08BD10B5074CA178601C94
:101A740000F0C2F8A178207103312046BDE810407F
:101A8400C9B200F0A1BE00BF0E00002070B581787D
:101A9400044643185A78013000F0C9F8C0B201284E
:101AA4000ED000231E4EA2785D1C0232DBB29A4295
:101AB4002FDA1C4800F05CFF22221B4B5A700FE007
:101AC4001122194D6A706278DD2A01D0EE2A07D1FD
:101AD400204600F031FBC0B2012801D122236B70F3
:101AE400114DA978681C00F087F828716378EE2BF3
:101AF40007D00A2B05D0A97828460331C9B200F0D3
:101B040063FE6378EE2B0AD1BDE87040074800F00D
:101B14002FBFE15C304600F0B7FE2B46C3E770BD33
:101B24000A3900081039000808000020213900088B
:101B3400002310B5C11C143011F8014F2344814215
:101B4400DBB2F9D19B1A5842584110BDC21C00F1B6
:101B54001403002012F8011F08449A42C0B2F9D1BC
:101B640070470000002310B50F4CC90007290FDC93
:101B740061B141F2210213F4004F4FEA43039BB2D7
:101B840001F1FF3118BF53400029F4D1184610BDAC
:101B940010F8012B083982EA132234F8122082EA61
:101BA40003239BB2E2E700BF14000020002330B5FA
:101BB400104DC900072911DC61B141F2210013F471
:101BC400004F4FEA43039BB201F1FF3118BF43407A
:101BD4000029F4D1981A18BF012030BD10F8014B28
:101BE400083984EA132435F8144084EA03239BB2A9
:101BF400E0E700BF1400002010B5FF230446221ABA
:101C0400D2B2914201D8184610BD14F8012B5340AA
:101C1400082213F0800F02F1FF324FEA430318BF8A
:101C240083F0310312F0FF02DBB2F2D1E7E730B503
:101C3400FF2305462C1AE4B2A14203D89B1A58424A
:101C4400584130BD15F8014B6340082413F0800F50
:101C540004F1FF344FEA430318BF83F0310314F057
:101C6400FF04DBB2F2D1E5E72DE9F04F814A91B0F0
:101C740005460C461068516804AB03C3127A0DF193
:101C840010091A700BAA90467B4B03F110071646F5
:101C940018685968083303C6BB423246F7D107AA0D
:101CA40017461B883380754B03F1080E16461868D7
:101CB4005968083303C673453246F7D118689B88C0
:101CC4003060B3800026DFF8F0A119F90620A35D87
:101CD4009A420AD06A4800F04BFE00232B806B80A6
:101CE40028462B7111B0BDE8F08F5046013600F044
:101CF4003FFE092EE9D1637A202BEBD1614800F035
:101D040037FEA37A002BE5D15F4800F031FEDFF8FF
:101D1400ACA104F10A0604F10D0916F8011F50469E
:101D240000F0B2FDB145F8D10026584A04F10E0A7C
:101D3400D34618F906909BF8001006F10E03894566
:101D44000AF1010A0DD04E48039300F011FE9BF8EE
:101D54000020314600924A46039B4D4800F094FD12
:101D6400BBE7104649460136039200F08DFD102E64
:101D7400039ADDD11E26454B04F11E09CA46BA1941
:101D840012F91E8C9AF80010A6F11E0B884509F171
:101D940001090AD03F4800F077FD9AF80030424626
:101DA4000093594633463C48D8E718464146013625
:101DB400039300F069FD2B2E039BDFD1DFF8008134
:101DC40004F12B0604F1310716F8011B404600F01C
:101DD4005BFDB742F8D13126304FA25D314638461B
:101DE400013600F051FD372EF7D194F837102C4806
:101DF40000F04AFD94F838102A4800F045FD94F8A4
:101E04003910284800F040FD94F83A10254800F0B5
:101E14003BFD94F83B10234800F036FD94F83C1049
:101E2400214800F031FD94F83D3094F83E603E21A5
:101E340006EB0326B6B232461C4800F025FD3246B6
:101E44003E211A4800F020FD94F83F3094F84040B9
:101E5400412104EB0324A4B22246154800F014FDEA
:101E640022464121134800F00FFD2E806C8001238F
:101E740036E700BF00390008A33A0008B53A000865
:101E84004C390008713900086C390008D139000850
:101E9400A7390008ED390008FC3900083C3A00086D
:101EA4005D3A0008613A0008683A0008713A00088F
:101EB400813A0008923A0008583900088539000828
:101EC400263A0008F8B501F1200323F0070300AF18
:101ED400ADEB030D04460D46FFF744FE0DEB050381
:101EE400020A9A750322D8751A761623F1228DF800
:101EF40000308DF801308DF802308DF80330002366
:101F04008DF80520A27968468DF80620E2798DF8CF
:101F140004308DF80720227A8DF811308DF80820CE
:101F2400627A6E468DF80920A27A8DF80A20E27A48
:101F34008DF80B20227B8DF80C20627B8DF80D2010
:101F4400A27B8DF80E20E27B8DF80F20227C8DF889
:101F540010208DF813308DF81450FFF7F7FD234649
:101F64008DF815001A1B954210DC731E621E06F1D3
:101F7400150113F8010F8B4202F8010FF9D1002368
:101F84000133042B06D12046BD46F8BD13F8012BBE
:101F94005A75E7E75A19A1183244527D4A75EFE79A
:101FA4002DE9F341857C014604466846FFF75CFE53
:101FB400A5F11003042B63D8DFE803F003173B48B3
:101FC40055000323E376002323776377A377E3772E
:101FD40084F8203084F8213090230C212046A37407
:101FE40002B0BDE8F041FFF76DBFE37EA17E1B04A4
:101FF40003EB0163617F244F0B44217F234D03EBEB
:1020040001233B6000232E68DFF88480A377E37705
:1020140084F8203084F821303B689E4202D32B6040
:102024009123DAE7A319197B404600F02DFC013611
:10203400F2E70323E376002323776377A377E37739
:1020440084F8203084F821309223C6E70323E37612
:10205400002323776377A377E37784F8203084F829
:1020640021309323B9E70323E376002323776377AF
:10207400A377E37784F8203084F821309423ACE705
:1020840002B0BDE8F08100BF9C020020A002002045
:1020940032390008B0B50D4A00AFD3690C4823F0BB
:1020A4001003D36100F064FC0A4B0B4A1B680B4C11
:1020B4000B481360236000F05BFC0A4B1B6883F33E
:1020C40008882368BD46BDE8B040184700100240A8
:1020D400DE3A000804500008480700204C0700209E
:1020E400F03A0008005000082DE9F0410546044686
:1020F40000270F4EDFF83C80AB78621B023B934213
:1021040002DC3846BDE8F0812379E278316802EBDD
:10211400032292B200230120FEF774FB18B140465B
:1021240000F026FC01273368023402333360E3E70E
:1021340014020020C33A000838B500230E4C0546AB
:1021440023600E4BA3601F23E360FEF715FB0C4BCB
:102154001A784AB901220B4920461A70FEF7BCFBD3
:1021640010B1094800F004FC2846FFF7BDFF0446FF
:10217400FEF714FB204638BDA402002000500008DE
:10218400B8020020B4020020CF3A00080268084BCD
:102194009A420BD1074A136801331360064A136845
:1021A40001331360054A136801331360704700BF9D
:1021B40000100040C4020020C0020020BC02002025
:1021C40010B514460A230248FFF722FA204610BD30
:1021D4002C08002010B590B02822002106A800F099
:1021E4004BFB1422002101A800F046FB01230A93B3
:1021F400102302240B934FF4401306A80F93069464
:102204000D94FEF72DFD0F234FF4806201930023FC
:10221400214601A80294039304920593FEF7E8FE75
:1022240010B010BD80B588B0FEF72AF8FFF7D2FFD2
:102234001022614D00210DEB020000F01DFBAB6983
:10224400002243F01003AB61AB694FF4004103F08B
:1022540010030193019BAB69584843F00803AB6139
:10226400AB69002403F008030293029BAB69534E4D
:1022740043F00403AB61AB6903F004030393039BD2
:10228400FEF764FC4FF400430493012305930223F7
:1022940004A94A4807930694FEF76CFB6B69484807
:1022A40043F001036B616B69464A03F00103009339
:1022B400009B4FF4E13380E80C000C2384604361FD
:1022C400C46004618461C461FFF774F93E483F4906
:1022D4003F4B846080E80A004FF48043C46003618C
:1022E40044618461C4610462FEF73AFC41F2DF5345
:1022F400384D3948AC6085E8090009232846EB606D
:10230400AC6104940594FFF743F804A928460494A7
:102314000594FFF757F8224621460F20FDF7E6FF04
:102324000F20FEF717F8224621462520FDF7DEFF91
:102334002520FEF70FF8224621463620FDF7D6FF6A
:102344003620FEF707F8224621460E20FDF7CEFF81
:102354000E20FDF7FFFF2846FEF71CFF1F4B21460A
:102364001B681F4D986800F00BFBFFF77DFB1D48B1
:1023740000F090F91C4C2368B3F5FA7F06D94FF4AA
:1023840000413046FEF7E7FB00232360154C0C4F59
:10239400A368002B02DD2B681E2B03D8134F40F6D5
:1023A400B83405E0384600F083F9F1E7FFF772FE30
:1023B4003B68A342FAD8DDE7001002400010014058
:1023C4002C0800200038014050070020005800402D
:1023D400801A06006C080020001000401C02002037
:1023E400C4020020AC080020C0020020BC0200206F
:1023F400704700000E4B82B09A6942F001029A6164
:102404009A6902F001020092009ADA6942F080525D
:10241400DA61DB69074A03F080530193019B536837
:1024240023F0E06343F00073536002B0704700BFD1
:10243400001002400000014010B5044686B010228E
:10244400002102A800F018FA2268114B9A421DD10B
:10245400104C02A9A369104843F00803A361A369BF
:1024640003F008030093009B4FF44063029312238C
:10247400039303230593FEF77DFAE36943F4800392
:10248400E361E36903F480030193019B06B010BD8B
:102494000058004000100240000C01400268084B44
:1024A40082B09A420AD103F50033DA6942F010028D
:1024B400DA61DB6903F010030193019B02B07047FA
:1024C4000010004070B5064686B01022002102A814
:1024D40000F0D2F932682B4B9A4251D103F558439C
:1024E4009A6902A942F480429A619A69264802F4E0
:1024F40080420092009A9A69002542F004029A618F
:102504009B69224C03F004030193019B4FF4007375
:1025140002930223039303230593FEF72BFA4FF44C
:102524008063194802A9029303950495FEF722FAE1
:10253400174B204684E828008023A560E3602561CA
:102544006561A561E561FDF727FF08B1FFF750FF5D
:102554004FF0100C0F4B746366620F4C802284E8BA
:10256400081000232046A360E26023616361A36135
:10257400E361FDF711FF08B1FFF73AFF34636662C8
:1025840006B070BD0038014000080140E807002093
:102594005800024044000240A40700207047FEE7B0
:1025A400FEE7FEE7FEE7704770477047FDF77ABE27
:1025B4000148FDF7DDBF00BFA40700200148FDF777
:1025C400D7BF00BFE80700200148FFF7A5B900BF47
:1025D4002C0800200148FEF7ECBD00BF6C08002069
:1025E40070B50E4615460C46A31B9D4201DC2846D9
:1025F40070BDAFF3008004F8010BF5E708B50A4B92
:102604000246196809B909491960694618680244FB
:102614008A4206D900F006F90C2303604FF0FF301C
:1026240008BD1A6008BD00BFC80200206011002068
:102634004FF0FF3070474FF4005300204B60704759
:1026440001207047002070470F4B1A6842F00102C6
:102654001A6059680D4A0A405A601A6822F0847256
:1026640022F480321A601A6822F480221A605A68AE
:1026740022F4FE025A604FF41F029A604FF0006287
:10268400034B9A60704700BF001002400000FFF83F
:1026940000ED00E0002301224360036083600249EF
:1026A4000248FFF74BB800BFB80800202C080020F0
:1026B4002B4A70B51068431C13602A4B596803F108
:1026C4000C040D5D284C0131255440F24B408142ED
:1026D400C8BF00219D685960013D9D607DB91560AA
:1026E4002378BE2B0CD12048FFF7D0F9002340F209
:1026F4004C42635501359542FBD11C4A136070BDB1
:102704002378162BF2D16378162BEFD1A378162BEE
:10271400ECD1E378162BE9D1627D12211248FFF740
:1027240007FAC8B1E37C217D114841EA032101F194
:10273400180201F11703E35CA65C46EA032632465D
:10274400FFF734FA18B10848FFF72AFCCEE7314600
:10275400084800F099F8C9E7617D0748F9E700BF28
:10276400CC020020AC080020D0020020BC020020D3
:10277400E60200200E3B00081C3B000800220E4B22
:1027840010B51A6040F24B420C4C2368013393425B
:10279400C8BF00232360A36801339342A36001DD13
:1027A400FFF786FF236806490122BDE8104019445B
:1027B4000448FEF7C3BF00BFC4020020AC080020D9
:1027C400B80800202C0800200A4601460148FEF7FC
:1027D4007BBF00BF2C080020002103E00B4B5B589B
:1027E400435004310A480B4B42189A42F6D30A4A22
:1027F40002E0002342F8043B084B9A42F9D3FFF766
:1028040023FF00F015F8FFF70DFD7047D03B0008DB
:1028140000000020800200208002002060110020BF
:10282400FEE70000014B1868704700BF1C0200203F
:1028340070B500250C4E0D4CA41BA410A54209D163
:1028440001F048F800250A4E0A4CA41BA410A54226
:1028540005D170BD56F8253098470135EEE756F896
:10286400253098470135F2E7C83B0008C83B00080B
:10287400C83B0008CC3B000803460244934200D105
:10288400704703F8011BF9E70FB40A4B13B51C6832
:1028940024B1A36913B9204600F0DAFA05AB049A0F
:1028A400A1682046019300F09BFC02B0BDE81040F3
:1028B40004B070471C02002070B50E46054618B1DE
:1028C40083690BB900F0C4FAAB69AC6813B9284644
:1028D40000F0BEFA234B9C4217D16C68A3891B07F6
:1028E4001DD52369DBB1013EA36816F8011F013B26
:1028F400A360E9B9002B2EDA22460A21284600F00B
:10290400F5F8013011D00A2070BD174B9C4201D15B
:10291400AC68E3E7154B9C4208BFEC68DEE7214650
:10292400284600F035F90028DDD04FF0FF3070BDA7
:10293400002B04DAA269934206DB0A2904D0236837
:102944005A1C22601970CFE72246284600F0CEF8C0
:102954000130C9D1E9E70A2023685A1C22601870A3
:1029640070BD00BF543B0008743B0008343B0008B2
:10297400024B01461868FFF79FBF00BF1C020020EE
:1029840000294FF480630CBF0222002200F000B83B
:102994002DE9F7431D46514B04461E680F469046E9
:1029A40026B1B36913B9304600F052FA4C4B9C423D
:1029B40052D17468B8F1020F06D0B8F1010F00F2D9
:1029C4008980002DC0F286802146304600F0D6F979
:1029D400616B41B104F14403994202D0304600F0E6
:1029E4002DFB002363630023A3616360A3891B069B
:1029F40003D52169304600F021FBA389B8F1020F09
:102A040023F44A6323F00303A3815DD001AB6A4638
:102A14002146304600F0A6FAA3891843A0812DBBB5
:102A2400009D284600F002FB074600284ED1DDF841
:102A34000090A9453CD14FF0FF30A38943F0020335
:102A4400A3810023A36004F14703236023610123CE
:102A5400636103B0BDE8F083224B9C4201D1B468AA
:102A6400A8E7214B9C4208BFF468A3E7002FD8D005
:102A7400B36913B9304600F0EBF9B8F1010F08BFA0
:102A8400A389276004BF43F00103A381A3892761BD
:102A940013F0080065611BD013F001004FF0000330
:102AA4001FBF6D42A360A561184608BFA560D0E7AB
:102AB400484600F0BBFA07460028BCD0A3894D461F
:102AC40043F08003A381D3E70020B6E7A946F5E7E6
:102AD400A060BEE74FF0FF30BBE700BF1C02002040
:102AE400543B0008743B0008343B0008F8B50E461C
:102AF4001446054618B183690BB900F0A9F9214BB6
:102B04009C422AD16C68A369A360A3891A072ED5B5
:102B1400236963B323692068F6B2C01A6369374630
:102B2400984204DB2146284600F028F928BBA36814
:102B34000130013BA36023685A1C22601E70636944
:102B4400984204D0A389DB0719D50A2E17D1214650
:102B5400284600F013F990B10FE00B4B9C4201D1D1
:102B6400AC68D0E7094B9C4208BFEC68CBE7214630
:102B7400284600F00DF80028CCD04FF0FF37384637
:102B8400F8BD00BF543B0008743B0008343B000808
:102B9400324B70B51D6806460C4625B1AB6913B9B6
:102BA400284600F055F92E4B9C420FD16C68B4F9BD
:102BB4000C309AB215072CD4D00611D409223260F5
:102BC40043F04003A3814FF0FF3070BD254B9C427E
:102BD40001D1AC68EBE7244B9C4208BFEC68E6E704
:102BE400510712D5616B41B104F14403994202D0FB
:102BF400304600F023FA00236363A38923F02403FF
:102C0400A3810023636023692360A38943F008033D
:102C1400A38123694BB9A38903F42073B3F5007F1F
:102C240003D02146304600F0C1F9A28912F0010315
:102C34000CD00023A36063695B42A361236953B989
:102C4400B4F90C3013F08000BAD170BD920758BFAC
:102C54006369A360F2E70020F7E700BF1C020020CD
:102C6400543B0008743B0008343B00088A892DE972
:102C7400F041054610070C465AD44B68002B05DC7E
:102C84000B6C002B02DC0020BDE8F081E66A002E0C
:102C9400F9D0002312F480522F682B6033D0606D7A
:102CA400A3895A0705D56368C01A636B0BB1236CFB
:102CB400C01A00230246E66A216A2846B047431C2C
:102CC400A38906D129681D294BD82B4ACA40D607A7
:102CD40047D5002262602269D904226004D5421CCF
:102CE40001D12B6803B96065616B2F600029CAD0DC
:102CF40004F14403994202D0284600F09FF90020D1
:102D04006063BDE8F081216A01232846B047411C75
:102D1400C6D12B68002BC3D01D2B01D0162B01D19B
:102D24002F60B0E7A38943F04003A381BDE8F0819D
:102D34000F69002FA7D0930718BF00230E6808BFA0
:102D44004B69A6EB07080F608B60B8F1000F9ADDA2
:102D540043463A46216A2846A66AB047002807DC5B
:102D6400A38943F04003A3814FF0FF30BDE8F08115
:102D74000744A8EB0008E8E70100402038B50B69D8
:102D840005460C46DBB118B183690BB900F060F855
:102D94000C4B9C4209D16C68B4F90C307BB12146D0
:102DA4002846BDE83840FFF761BF074B9C4201D17C
:102DB400AC68F1E7054B9C4208BFEC68ECE70020E7
:102DC40038BD00BF543B0008743B0008343B000886
:102DD400014900F0A9B800BF812D0008002310B5F7
:102DE400044603604360836081814366C28103615A
:102DF40043618361194608225C30FFF73DFD054BB2
:102E040024626362044BA362044BE362044B2363B6
:102E140010BD00BF6137000883370008BB370008C6
:102E2400DF37000870B568254A1E55430E4605F184
:102E3400740100F04FF9044640B1002180E84200DB
:102E44000C30A06005F16802FFF716FD204670BD46
:102E5400836910B5044633BB8364C3640365124BB2
:102E6400124A1B688262984204BF0123836100F006
:102E74001FF86060204600F01BF8A060204600F0B8
:102E840017F80022E06004216068FFF7A7FF012221
:102E94000921A068FFF7A2FF02221221E068FFF7D0
:102EA4009DFF0123A36110BD303B0008D52D000810
:102EB400F8B51C4B07461E68B36913B93046FFF7D3
:102EC400C7FF4836B4687368013B03D5336833B130
:102ED4003668F7E7B4F90C506DB16834F4E70421AF
:102EE4003846FFF79FFF30600028F1D10C230446D9
:102EF4003B602046F8BD4FF6FF73E381012365660E
:102F0400A3812560A560656025616561A5610822CE
:102F1400294604F15C00FFF7AFFC6563A563A56473
:102F2400E564E6E7303B00082DE9F843804689462E
:102F3400002600F1480414B93046BDE8F883A568BA
:102F44006768013F01D52468F5E7AB89012B07D9F0
:102F5400B5F90E30013303D029464046C84706432D
:102F64006835EEE770B50E46B1F90E1090B0002941
:102F740014461D4607DA00232B60B3891A0610D4C1
:102F84004FF480630EE001AA00F04EFC0028F2DB4F
:102F9400029A02F47042A2F500535A425A412A603E
:102FA400EEE740230020236010B070BD8B8973B519
:102FB4009D0706460C4607D504F1470323602361A9
:102FC4000123636102B070BD01AB6A46FFF7CAFF1B
:102FD40000990546304600F07DF848B9B4F90C3044
:102FE4009A05EFD423F0030343F00203A381E3E73C
:102FF4000D4BB362A389206043F08003A381009B3F
:1030040020616361019B5BB1B4F90E10304600F09E
:103014001DFC28B1A38923F0030343F00103A3811A
:10302400A3891D43A581CDE7D52D0008024B014698
:10303400186800F04FB800BF1C02002038B50546E0
:10304400002943D051F8043C0C1F002BB8BFE418EE
:1030540000F02CFC1E4A1368104633B963601460F8
:103064002846BDE8384000F022BCA3420BD92168B1
:103074006218934201BF1A685B6852182260636049
:103084000460EDE713465A680AB1A242FAD91968F6
:103094005818A0420BD12068014458188242196084
:1030A400DED110685268014419605A60D8E702D929
:1030B4000C232B60D4E7206821188A4201BF1168D1
:1030C40052680918216062605C60C9E738BD00BFBE
:1030D4001C07002070B5CD1C25F0030508350C2D08
:1030E40038BF0C25002D064601DBA94203D90C2369
:1030F4003360002070BD00F0D9FB234A14682146D8
:1031040091B9224C23681BB9304600F017FB2060AC
:103114002946304600F012FB431C26D10C233046CE
:10312400336000F0C4FBE4E70B685B1B1AD40B2B81
:103134000FD90B60CC18CD50304600F0B8FB04F129
:103144000B00231D20F00700C31A1BD05A42E25083
:1031540070BD8C420BBF63684B681360636018BF1B
:103164000C46E9E70C464968CAE7C41C24F003048A
:10317400A04205D0211A304600F0E0FA0130CDD04B
:103184002560D9E770BD00BF1C0700202007002080
:10319400936810B4013B002B936008DA9469A3424E
:1031A40002DBCBB20A2B02D110BCFFF79FBC136821
:1031B400581C10601970C8B210BC7047F8B50646A8
:1031C4000F461446D518AC4201D1002007E03A4618
:1031D40014F8011B3046FFF7DBFF431CF3D1F8BDA5
:1031E4002DE9F04F9DB00C4617460393064618B1DF
:1031F40083690BB9FFF72CFE7C4B9C4257D1746852
:10320400A38918075DD52369002B5AD0002309939D
:1032140020238DF8293030234FF0010B8DF82A300C
:10322400B846454615F8013B002B55D1B8EB070AC3
:103234000BD053463A4621463046FFF7BFFF0130D4
:1032440000F0C480099B5344099398F80030002B84
:1032540000F0BC8000234FF0FF32049307930592E3
:1032640006938DF853301A9305222978604800F0AC
:103274000FFB05F10108049B002831D1D90644BF96
:1032840020228DF853201A0744BF2B228DF8532097
:103294002A782A2A2CD000210A20079AA84698F8CE
:1032A40000300135303B092B6DD971B326E0514B09
:1032B4009C4201D1B468A3E74F4B9C4208BFF46819
:1032C4009EE721463046FFF763FC00289ED04FF06E
:1032D400FF301DB0BDE8F08F252BA7D0A846A0E78E
:1032E400434A4546801A0BFA00F018430490BBE7A2
:1032F400039A111D12680391002A01DB079204E06E
:10330400524243F002030792049398F800302E2BA4
:1033140010D198F8013008F101012A2B37D1039B11
:1033240008F102081A1D1B680392002BB8BF4FF066
:10333400FF330593314D032298F80010284600F01E
:10334400A7FA40B14023401B03FA00F0049B08F1A4
:1033540001080343049398F800100622284808F152
:1033640001078DF8281000F093FA002834D0254B7B
:1033740003BB039B073323F0070308330393099B21
:103384004B4409934CE700FB0232012186E70023FA
:103394000A2518460593884698F800200131303AEA
:1033A400092A03D9002BC5D00590C3E705FB0020EB
:1033B4000123F0E703AB00932246134B04A93046E4
:1033C400AFF30080B0F1FF3F8146D8D1A3895B06FB
:1033D4003FF57DAF09987CE703AB009322460A4B87
:1033E40004A9304600F08AF8ECE700BF543B00081B
:1033F400943B0008743B0008343B00089A3B0008E7
:103404009E3B000800000000C13100082DE9F04790
:1034140091461F468A680B6906469342B8BF134615
:10342400C9F8003091F843200C46DDF8208012B131
:103434000133C9F800302368990642BFD9F8003037
:103444000233C9F80030256815F0060507D104F1E8
:10345400190AE368D9F800209B1A9D422ADB94F8E4
:1034640043302268003318BF012392062FD404F19D
:10347400430239463046C047013022D02368E5680C
:1034840003F00603042B18BF0025D9F800204FF0E1
:10349400000908BFAD1AA368226908BF25EAE575CB
:1034A4009342C4BF9B1AED181A344D451BD100201A
:1034B400BDE8F0870123524639463046C047013003
:1034C40003D14FF0FF30BDE8F0870135C1E730206C
:1034D400E11881F843005A1C94F845102244023341
:1034E40082F84310C3E70123224639463046C047D9
:1034F4000130E6D009F10109D7E700002DE9F043D6
:1035040017460A7E85B06E2A984606460C460C9BE2
:1035140001F1430E00F0BC801AD8632A2ED00AD8D9
:10352400002A00F0C880582A00F08A8004F142057D
:1035340084F842202AE0642A01D0692AF6D121685D
:103544001A6811F0800F23D0111D1960136827E049
:10355400732A00F0B48008D86F2A2AD0702AE5D1E3
:103564000A6842F020020A6003E0752A21D0782A12
:10357400DCD178226F4984F8452064E01A6801F1AF
:103584004205111D1960136884F842300123A3E039
:1035940011F0400F02F104011960D7D0B2F90030E4
:1035A400002B03DA2D225B4284F8432062490A226D
:1035B40017E02068196810F0800F03D0081D186008
:1035C4000B6806E010F0400F01F104001860F7D01A
:1035D4000B886F2A14BF0A2208225749002084F856
:1035E40043006568002DA560C0F29C80206820F02F
:1035F40004002060002B3FD1002D40F095807546DB
:10360400082A0BD12368DA0708D5236962689A422D
:10361400DEBF302305F8013C05F1FF35AEEB0503B1
:103624002361CDF800803B4603AA21463046FFF7CC
:10363400EDFE013055D14FF0FF3005B0BDE8F08309
:1036440081F845203C492268186812F0800F00F187
:1036540004051D6001D0036802E05506FBD503880C
:10366400D00744BF42F0200222601BB9226822F036
:10367400200222601022B1E77546B3FBF2F002FB90
:103684001033CB5C05F8013D03460028F5D1B7E7BC
:1036940008681A6810F0800F496904D0101D18607A
:1036A4001368196007E010F0400F02F1040018607D
:1036B4001368F6D01980002375462361B1E71A68B0
:1036C400111D1960156800216268284600F0E0F8B1
:1036D40008B1401B606063682361002384F84330B1
:1036E4009FE723692A4639463046C0470130A2D0B5
:1036F40023689B0707D5002504F11909E368039A99
:103704009B1A9D4205DBE068039B9842B8BF1846AC
:1037140093E701234A4639463046C04701308AD0F0
:103724000135EBE7002BA7D10B7804F1420584F8AF
:10373400423065E7B63B0008A53B000838B50023D6
:10374400054C054608462360FEF758FF431C02D18A
:10375400236803B12B6038BD5C11002010B50C4602
:10376400B1F90E1000F0A4F80028ABBF636DA38973
:103774001B1823F48053ACBF6365A38110BD2DE9EE
:10378400F0411F468B890546DB050C46164605D5D8
:1037940002230022B1F90E1000F068F8A389324622
:1037A40023F48053A381B4F90E103B462846BDE8A8
:1037B400F04100F017B810B50C46B1F90E1000F046
:1037C40055F8431CA38915BF606523F4805343F463
:1037D4008053A38118BFA38110BDB1F90E1000F06E
:1037E40013B8000038B50546084611460022054CBA
:1037F40022601A46FEF7E4FC431C02D1236803B19D
:103804002B6038BD5C11002038B50023054C0546FB
:1038140008462360FEF70CFF431C02D1236803B162
:103824002B6038BD5C11002038B50023064C0546DA
:10383400084611462360FEF7FEFE431C02D12368AE
:1038440003B12B6038BD00BF5C11002038B50023E4
:10385400054C054608462360FEF7F2FE431C02D1E0
:10386400236803B12B6038BD5C11002038B50546D0
:10387400084611460022054C22601A46FEF7E2FE75
:10388400431C02D1236803B12B6038BD5C110020B6
:1038940010B5C9B202449042034601D1002010BDC4
:1038A4001C7801308C42F6D1184610BD7047704721
:1038B40038B50546084611460022054C22601A46D2
:1038C400FEF78EFE431C02D1236803B12B6038BD82
:1038D4005C110020F8B500BFF8BC08BC9E467047D8
:0C38E400F8B500BFF8BC08BC9E46704759
:1038F00002030405060708090A0B0C0D0E0F101031
:103900004A542D4E52444153200025303278200035
:10391000436865636B2053756D206572726F72200A
:103920000075706461746520436F6D706C657465BB
:1039300020004D4249435F446F776E4C6F61644491
:103940006174615B695D203A20257800446174618F
:103950002044696666200D004D41524B204461743D
:10396000612053756363657373200D0046696C6550
:1039700020547970652044617461205375636365D8
:103980007373200D0056657273696F6E2044617405
:103990006120537563636573732056657273696F35
:1039A0006E2025780D0A004D4249435F46696C65DB
:1039B0004E616D65315B25645D203A2025782C20B1
:1039C000646174615B25645D203A202025780D0ACE
:1039D0000046696C65204E616D652044617461200C
:1039E000537563636573732025630D0A0044617426
:1039F0006120446966662025630D0A004D424943F3
:103A00005F46696C654E616D65325B25645D203A89
:103A10002025782C20646174615B25645D203A2048
:103A20002025780D0A004372656174696F6E20531A
:103A30007563636573732025780D0A0043726561B1
:103A400074696F6E2053756363657373206461746A
:103A5000615B25645D203A2025780D0A00202564ED
:103A600000202D2530326400202D253032640D0ACF
:103A700000646174615B25645D203A2025640D0A51
:103A8000004352435F485B25645D203A2025780D52
:103A90000A004352435F4C5B25645D203A20257841
:103AA0000D0A006A6866732D6D6269632D6E72641B
:103AB00061732D76007630302E30302E30312E6D01
:103AC00062630048414C204E4F54204F4B2000452C
:103AD00072617365204661696C6564200D00626FD8
:103AE0006F74206C6F61646572207374617274000E
:103AF0006A756D70210000000000000000000102E6
:103B000003040607080900000000010203044352F1
:103B10004320455252202578200D0A004348454352
:103B20004B2053554D20455252202578200D0A0038
:103B30002002002000000000000000000000000043
:103B40000000000000000000000000000000000075
:103B50000000000000000000000000000000000065
:103B60000000000000000000000000000000000055
:103B70000000000000000000000000000000000045
:103B80000000000000000000000000000000000035
:103B900000000000232D302B2000686C4C0065666F
:103BA000674546470030313233343536373839418E
:103BB00042434445460030313233343536373839A4
:083BC0006162636465660000A8
:043BC80009020008E6
:043BCC00E501000807
:103BD0000100000010000000BE11030500BEBE0B76
:103BE000030400EB00002110422063308440A55004
:103BF000C660E770088129914AA16BB18CC1ADD133
:103C0000CEE1EFF13112100273325222B5529442DA
:103C1000F772D662399318837BB35AA3BDD39CC382
:103C2000FFF3DEE36224433420040114E664C77426
:103C3000A44485546AA54BB528850995EEE5CFF5D2
:103C4000ACC58DD55336722611163006D776F6667A
:103C50009556B4465BB77AA719973887DFF7FEE722
:103C60009DD7BCC7C448E5588668A7784008611846
:103C700002282338CCC9EDD98EE9AFF94889699972
:103C80000AA92BB9F55AD44AB77A966A711A500A1A
:103C9000333A122AFDDBDCCBBFFB9EEB799B588BC2
:103CA0003BBB1AABA66C877CE44CC55C222C033C66
:103CB000600C411CAEED8FFDECCDCDDD2AAD0BBD12
:103CC000688D499D977EB66ED55EF44E133E322EBA
:103CD000511E700E9FFFBEEFDDDFFCCF1BBF3AAF62
:103CE000599F788F8891A981CAB1EBA10CD12DC1C0
:103CF0004EF16FE18010A100C230E3200450254056
:103D000046706760B9839893FBA3DAB33DC31CD3B5
:103D10007FE35EF3B1029012F322D23235421452A5
:103D200077625672EAB5CBA5A89589856EF54FE501
:103D30002CD50DC5E234C324A014810466744764F5
:103D400024540544DBA7FAB79987B8975FE77EF755
:103D50001DC73CD7D326F2369106B0165766767645
:103D6000154634564CD96DC90EF92FE9C899E98921
:103D70008AB9ABA94458654806782768C018E10895
:103D80008238A3287DCB5CDB3FEB1EFBF98BD89BF5
:103D9000BBAB9ABB754A545A376A167AF10AD01AE5
:103DA000B32A923A2EFD0FED6CDD4DCDAABD8BAD41
:103DB000E89DC98D267C076C645C454CA23C832C35
:103DC000E01CC10C1FEF3EFF5DCF7CDF9BAFBABF95
:103DD000D98FF89F176E367E554E745E932EB23E85
:103DE000D10EF01E0050000800A24A04200200205C
:103DF00000000000543B0008743B0008343B0008FE
:103E000000000000000000000000000000000000B2
:103E100000000000000000000000000000000000A2
:103E20000000000000000000000000000000000092
:103E30000000000000000000000000000000000082
:103E40000000000000000000000000000000000072
:04000005080027DDEB
:00000001FF
